:020000040000FA
:100000000C946E010C9496010C9496010C9496013C
:100010000C9496010C9496010C9496010C94960104
:100020000C9496010C9496010C94F6040C947D05A6
:100030000C9496010C9496010C9496010C949601E4
:100040000C9496010C9496010C9496010C949601D4
:100050000C9496010C9496010C9496010C94B501A5
:100060000C9496010C9496010C9496010C949601B4
:100070000C9496010C9496010C9496010C949601A4
:100080000C9496010C9496010C9496010C94960194
:100090000C9496010C9496010C9496010C94960184
:1000A0000C9496010C9496010C94960100000000AB
:1000B000240027002A002D00300000000000250049
:1000C00028002B002E003100000000002300260035
:1000D00029002C002F000404040404030405020278
:1000E00002020403020202020606060606060404D1
:1000F00002020204040802011040804010204080E7
:10010000408008020401804020100201108010206D
:1001100040400000000200080E0000030401000B34
:100120000000070605040100080A0B0C0D09040372
:1001300009042203410072006400750069006E002A
:100140006F0020004C0065006F006E0061007200BF
:1001500064006F00180341007200640075006900BC
:100160006E006F0020004C004C00430012010002A2
:10017000000000404123368000010102000112010D
:10018000000202000040412336800001010200010C
:1001900000C18081C1080B000202020100090400B5
:1001A00000010202000005240010010524010101E4
:1001B00004240206052406000107058103100040FF
:1001C00009040100020A00000007050202400000C5
:1001D0000705830240000005010902A1010901A1F0
:1001E00000850105091901290315002501950375ED
:1001F0000181029501750581030501093009310965
:10020000381581257F750895038106C0C005010951
:1002100006A1018502050719E029E71500250175EA
:1002200001950881029501750881039506750815E9
:100230000025650507190029658100C00904020031
:1002400001030000000921010100012265000705EA
:10025000840340000100000000000000002A2B2859
:10026000000000000000000000000000000000008E
:1002700000000000002C9EB4A0A1A2A434A6A7A553
:10028000AE362D3738271E1F20212223242526B3E2
:1002900033B62EB7B89F8485868788898A8B8C8DE4
:1002A0008E8F909192939495969798999A9B9C9DF6
:1002B0002F3130A3AD350405060708090A0B0C0DD4
:1002C0000E0F101112131415161718191A1B1C1DD6
:1002D000AFB1B0B5000032041007150811241FBEDD
:1002E000CFEFDAE0DEBFCDBF11E0A0E0B1E0E0EAA1
:1002F000F2E102C005900D92AC32B107D9F711E0DE
:10030000ACE2B1E001C01D92AD39B107E1F712E0F6
:10031000CCEDD2E004C02297FE010E944A09C63DFE
:10032000D107C9F70E946C030C944E090C9400008D
:100330008091000161E00E94390368EE73E080E083
:1003400090E00E94FD018091000160E00E9439036D
:1003500068EE73E080E090E00E94FD0108958091D6
:10036000000161E00E94AC0208951F920F920FB647
:100370000F9211242F933F938F939F93AF93BF932B
:100380008091300190913101A0913201B0913301FF
:10039000309134010196A11DB11D232F2D5F2D3702
:1003A00020F02D570196A11DB11D2093340180939B
:1003B000300190933101A0933201B09333018091C9
:1003C0002C0190912D01A0912E01B0912F01019649
:1003D000A11DB11D80932C0190932D01A0932E019E
:1003E000B0932F01BF91AF919F918F913F912F912A
:1003F0000F900FBE0F901F9018959B01AC017FB717
:10040000F89480912C0190912D01A0912E01B09132
:100410002F0166B5A89B05C06F3F19F00196A11D7D
:10042000B11D7FBFBA2FA92F982F8827860F911D46
:10043000A11DB11D62E0880F991FAA1FBB1F6A95FD
:10044000D1F7BC012DC0FFB7F89480912C01909199
:100450002D01A0912E01B0912F01E6B5A89B05C0FA
:10046000EF3F19F00196A11DB11DFFBFBA2FA92FB3
:10047000982F88278E0F911DA11DB11DE2E0880FD6
:10048000991FAA1FBB1FEA95D1F7861B970B885EA1
:100490009340C8F2215030404040504068517C4F5A
:1004A000211531054105510571F60895789484B5FB
:1004B000826084BD84B5816084BD85B5826085BD60
:1004C00085B5816085BDEEE6F0E080818160808346
:1004D000E1E8F0E010828081826080838081816029
:1004E0008083E0E8F0E0808181608083E1E9F0E0F2
:1004F000808182608083808181608083E0E9F0E098
:10050000808181608083E1ECF0E080818460808381
:10051000808182608083808181608083E3ECF0E071
:10052000808181608083E0ECF0E080818260808364
:10053000E2ECF0E0808181608083EAE7F0E0808196
:1005400084608083808182608083808181608083F9
:100550008081806880830895CF93DF93482F50E097
:10056000CA018C509F4FFC0134914A525F4FFA01EF
:100570008491882369F190E0880F991FFC01E4556C
:10058000FF4FA591B491FC01E654FF4FC591D49162
:10059000662351F42FB7F8948C91932F909589236B
:1005A0008C93888189230BC0623061F42FB7F89453
:1005B0008C91932F909589238C938881832B8883AA
:1005C0002FBF06C09FB7F8948C91832B8C939FBF4D
:1005D000DF91CF910895883071F1893068F48230CD
:1005E00031F1833020F4813009F042C01DC08330E6
:1005F00089F08430E9F512C08B3059F18C3028F441
:100600008930E9F08A30A1F51EC08C3031F18E308E
:1006100079F529C0809180008F7703C08091800098
:100620008F7D80938000089584B58F7702C084B554
:100630008F7D84BD0895809190008F7707C0809151
:1006400090008F7D03C080919000877F8093900001
:1006500008958091C0008F7703C08091C0008F7D86
:100660008093C00008958091C200877F8093C2006C
:100670000895FF920F931F93F62E482F50E0CA0162
:100680008E5E9E4FFC012491CA018C509F4FFC014D
:1006900014914A525F4FFA0104910023C9F02223BA
:1006A00019F0822F0E94EB02E02FF0E0EE0FFF1F07
:1006B000E654FF4FA591B4919FB7F894FF2021F421
:1006C0008C911095812302C08C91812B8C939FBFBC
:1006D0001F910F91FF900895CF93DF930E945602D0
:1006E0008DE391E00E9433040E94AF01C0E0D0E0AE
:1006F0000E9498012097E1F30E940000F9CF282F73
:10070000809137018823C1F057FF1AC015C028987F
:10071000909336018091F1008193E217F307B9F7C6
:100720004115510539F08091F200882319F48BE6C8
:100730008093E800AFBF02C04FEF5FEFCA0108959A
:10074000AFB7F89427702093E9008091F200282F2A
:1007500030E0241735070CF4A901FB019B01240F9D
:10076000311D94E6DACFDF93CF930F92CDB7DEB78A
:10077000BE016F5F7F4F41E050E00E947F03019711
:1007800019F02FEF3FEF03C08981282F30E0C90116
:100790000F90CF91DF910895FF920F931F93F82E42
:1007A000142F052F40913A0150913B01212F302FFA
:1007B000C901DC01FB016EEF29C0F7FE02C0949174
:1007C00001C09081209138013091390124173507FB
:1007D000ACF48091E8008570E1F38091E80082FF3D
:1007E00003C02FEF3FEF17C09093F100C9010196AE
:1007F0008F739070892B11F46093E8002F5F3F4F47
:100800003093390120933801119731961097A9F64A
:10081000812F902F9C01C9011F910F91FF90089586
:100820009C018091E80082FFFCCFF901260F311D69
:1008300003C08091F1008193E217F307D1F7289864
:1008400084E6809336018BEF8093E800CB01089516
:100850008093E9008091F200882319F08AE3809365
:10086000E800089508951092370181E08093D70041
:1008700080EA8093D80082E189BD09B400FEFDCFF3
:1008800061E070E080E090E00E94FD0180E98093EB
:10089000D8008CE08093E2001092E000559A209AF4
:1008A00008955F926F927F928F929F92AF92BF92C4
:1008B000CF92DF92EF92FF920F931F93CF93DF932C
:1008C000E82E842E752E80913701882371F18B01DB
:1008D000242F352FC901EC017AEFF72E67E0962E11
:1008E0009E2050E4552E8E2D90E040E2A42EB12C97
:1008F000A822B9223AE3632E20E4C22ED12CC822CA
:10090000D92258C09FB7F8949092E9008091E800EE
:1009100085FD02C020E004C08091F200252D281B37
:100920009FBF222361F4FA9419F42FEF3FEF4DC0DB
:1009300061E070E080E090E00E94FD013BC0822F0A
:1009400090E0C817D9070CF42C2FC21BD1094FB760
:10095000F8949092E900A114B10421F406C0109219
:10096000F10021502223D9F719C0E7FC03C0F80198
:10097000922F10C0C801322F06C0FC010196E491ED
:10098000E093F10031503323C1F706C08191809389
:10099000F10091509923D1F7020F111D8091E800C9
:1009A00085FF05C0209729F4C114D10411F060928D
:1009B000E8004FBF209709F0A5CF5D9884E68093AB
:1009C0003501282D372DC9019C01C901DF91CF9137
:1009D0001F910F91FF90EF90DF90CF90BF90AF905D
:1009E0009F908F907F906F905F9008951F920F92CD
:1009F0000FB60F9211242F933F934F935F936F93F2
:100A00007F938F939F93AF93BF93EF93FF938091C7
:100A1000E1001092E100982F83FF0FC01092E900CF
:100A200081E08093EB001092EC0082E38093ED0074
:100A30001092370188E08093F00092FF34C083E089
:100A40008093E9008091F200882319F08AE3809373
:100A5000E8008FB7F89492E09093E9009091F2004B
:100A60008FBF992321F082E891E00E945307809183
:100A70003501882351F080913501815080933501F3
:100A800080913501882309F45D9A8091360188238D
:100A900051F080913601815080933601809136016A
:100AA000882309F4289AFF91EF91BF91AF919F910C
:100AB0008F917F916F915F914F913F912F910F9007
:100AC0000FBE0F901F9018950F931F93DF93CF9336
:100AD0000F92CDB7DEB719828E010F5F1F4FC8018D
:100AE0000E947907C8010E941209898190E00F9045
:100AF000CF91DF911F910F9108951F920F920FB622
:100B00000F921124EF92FF921F932F933F934F93D5
:100B10005F936F937F938F939F93AF93BF93EF9365
:100B2000FF93DF93CF93CDB7DEB76197DEBFCDBF25
:100B30001092E9008091E80083FF0FC1FE01319619
:100B40009E01275F3F4F03C08091F1008193E21720
:100B5000F307D1F7289884E68093360182EF8093DB
:100B6000E800998197FF05C08091E80080FFFCCFE5
:100B700003C08EEF8093E800292F30E0C901807612
:100B80009070892B09F0C2C08A81882329F41092C1
:100B9000F1001092F100D6C0813009F4D3C0833047
:100BA00009F4D0C0853049F48091E80080FFFCCF83
:100BB0008B8180688093E300C5C0863009F07CC0DB
:100BC0001C81EF80F8841230C1F51092E900109278
:100BD00039011092380110923B0110923A010E94A3
:100BE000640599E0FE013996DF01292F1D922A95AF
:100BF000E9F799871A8791E09E8790E8988B9AEF9A
:100C0000998B2091380130913901275F3F4F3C8704
:100C10002B878D871092E9001092390110923801CC
:100C2000F0923B01E0923A0180E0BF0149E050E0E0
:100C30000E94CC030E94640585C01092E9001092C6
:100C4000390110923801F0923B01E0923A011232E0
:100C500041F482E290E00E940A09892B09F476C0EF
:100C600071C0113079F488E0E816F10419F481E0DC
:100C700080933C0180913C01882309F06BC0ECE635
:100C8000F1E013C0133009F061C08B81882319F49F
:100C9000EEE2F1E00AC0823019F4E2E3F1E005C0CF
:100CA000813009F053C0E4E5F1E0449180E8BF01F0
:100CB00050E00E94CC0346C0873009F447C088301A
:100CC00021F481E08093F1003DC08930D9F5237093
:100CD0003070232BD9F5E1E9F1E091E031E026E332
:100CE0009093E9003093EB0084918093EC00209383
:100CF000ED009F5F3196953099F78EE78093EA007B
:100D00001092EA008B81809337011CC08F819885F7
:100D10001092E900109239011092380190933B0132
:100D200080933A018D81882329F4CE0101960E9497
:100D3000850706C0823051F4CE0101960E94DB0780
:100D4000882321F08EEF8093E80007C081E2809332
:100D5000EB0003C0EEE7F1E0A8CF6196DEBFCDBFA8
:100D6000CF91DF91FF91EF91BF91AF919F918F91C3
:100D70007F916F915F914F913F912F911F91FF90C4
:100D8000EF900F900FBE0F901F90189520917E014D
:100D900030917F018091800190918101281B390B56
:100DA0002F733070C901089520917E0130917F0129
:100DB00080918001909181012817390719F42FEF54
:100DC0003FEF09C0E0918001F0918101E25CFE4FAC
:100DD0008081282F30E0C901089520917E01309153
:100DE0007F0180918001909181012817390719F4C2
:100DF0002FEF3FEF13C0E0918001F0918101E25CA1
:100E0000FE4F2081809180019091810101968F7326
:100E10009070909381018093800130E0C901089522
:100E2000109285011092840188EE93E0A0E0B0E07A
:100E30008093860190938701A0938801B0938901E4
:100E400080E191E0909383018093820108950F9354
:100E50001F93DF93CF930F92CDB7DEB78C016983D9
:100E600080910901882369F083E0BE016F5F7F4FA5
:100E700041E050E00E9451041816190614F49C0138
:100E800007C081E090E0F8019383828320E030E0A6
:100E9000C9010F90CF91DF911F910F91089583E0C9
:100EA0000E9428040895CF93DF9312C082E00E942D
:100EB000B3032FEF8F3F9207C9F0E0917E01F091CD
:100EC0007F01E25CFE4F8083D0937F01C0937E015F
:100ED000C0917E01D0917F012196CF73D070809117
:100EE000800190918101C817D90701F7DF91CF9157
:100EF0000895FC0180818E5F808380E865E971E060
:100F000042E450E00E94CC030895FC01818190816D
:100F1000913A59F4813209F04CC080E062E071E00E
:100F200047E050E00E94CC0342C0913209F041C03A
:100F3000803239F482E091E067E070E00E941004B2
:100F400036C0823209F035C08281809309018091D8
:100F5000020190910301A0910401B0910501805B11
:100F60009440A040B04019F58091090180FD12C065
:100F700087E797E790930108809300082BE088E1CA
:100F800090E00FB6F894A895809360000FBE209370
:100F900060000DC088E10FB6F89480936000109255
:100FA00060000FBEA895109201081092000881E021
:100FB000089580E00895FC0191818081813A31F4A7
:100FC000913089F080E0933089F40DC0813269F46A
:100FD0009B3021F4828180930A0105C09A3029F464
:100FE000828180930B0181E0089580E00895EF9263
:100FF000FF920F931F938C01E62EDC01ED91FC9183
:101000000480F581E02D0995F82ED801ED91FC9131
:101010000680F781E02DC8016E2D09958F2D90E097
:101020001F910F91FF90EF900895109290011092F0
:1010300094011092930182E291E090939201809347
:1010400091010895EF92FF920F931F93DF93CF9337
:101050000F92CDB7DEB789838B017A0184E0BE01A0
:101060006F5F7F4F41E050E00E94510484E4B8017B
:10107000A7010E9451040F90CF91DF911F910F9112
:10108000FF90EF90089582E048E050E00E9422082F
:101090000895FC0116821782108611861286138627
:1010A00014823496BF010E9443080895DC01683819
:1010B00010F0685829C0E62FF0E067FF13C0E05831
:1010C000F04081E090E002C0880F991FEA95E2F7B6
:1010D000809514962C911497282314962C9314978A
:1010E00060E012C0EB5AFD4F6491662319F420E0D2
:1010F00030E01DC067FF08C014968C9114978D7F57
:1011000014968C9314976F77FD0190E0662321F07D
:101110008681861709F416829F5F31969630B1F763
:10112000CD011496BD010E94430821E030E0C901C1
:101130000895CF93DF93DC01683810F0685825C01C
:10114000E62FF0E067FF12C0E058F04081E090E049
:1011500002C0880F991FEA95E2F714962C91149714
:10116000282B14962C93149760E00FC0EB5AFD4F78
:1011700064916623D9F167FF08C014968C91149787
:10118000826014968C9314976F7716968C911697AD
:101190008617A9F117968C911797861781F11896E3
:1011A0008C911897861759F119968C911997861773
:1011B00031F11A968C911A97861709F11B968C912A
:1011C0001B978617E1F0ED01E0E0F0E09E2F8E81A5
:1011D000882321F4EA0FFB1F668306C09F5F3196C8
:1011E0002196E630F10591F7963049F481E090E0E0
:1011F00013969C938E93129720E030E007C0CD01A8
:101200001496BD010E94430821E030E0C901DF913E
:10121000CF91089580E867ED71E045E650E00E94C7
:10122000CC030895FC0180818F5F808380E86CE3AC
:1012300072E049E150E00E94CC030895CF92DF9222
:10124000EF92FF920F931F93CF93DF937C016B017B
:101250008A01C0E0D0E00FC0D6016D916D01D701C9
:10126000ED91FC910190F081E02DC7010995C80F27
:10127000D91F015010400115110571F7CE01DF9102
:10128000CF911F910F91FF90EF90DF90CF90089535
:10129000EE0FFF1F0590F491E02D0994F894FFCF15
:1012A0000D0000E10000000000000101000000004E
:1012B00027071E09C606ED06D4064F075307000090
:1012C0000000F7071E09990856084908FFFFFFFFAD
:1012D000FFFFFFFFFFFFFFFFFFFFFFFFFFFFFFFF1E
:1012E000FFFFFFFFFFFFFFFFFFFFFFFFFFFFFFFF0E
:1012F000FFFFFFFFFFFFFFFFFFFFFFFFFFFFFFFFFE
:10130000FFFFFFFFFFFFFFFFFFFFFFFFFFFFFFFFED
